:100000000EC028C027C026C025C024C023C022C0DF
:1000100021C020C01FC01EC01DC01CC01BC0112499
:100020001FBECFE5D2E0DEBFCDBF10E0A0E6B0E05E
:10003000E0EDFCE102C005900D92A238B107D9F7BE
:1000400011E0A2E8B0E001C01D92AB31B107E1F7C9
:10005000E9D93DCED5CF89E288BB089520917700BC
:10006000309178004091790050917A00A7DD20E02E
:1000700030E040E050E004C02F5F3F4F4F4F5F4FF4
:100080006217730784079507BCF72093D500309358
:10009000D6004093D7005093D800089589E288BBDA
:1000A00061E070E080E090E0D9DF88E288BB0895ED
:1000B00020917B0030917C0040917D0050917E002A
:1000C0007DDD20E030E040E050E004C02F5F3F4F96
:1000D0004F4F5F4F6217730784079507BCF7209354
:1000E000D9003093DA004093DB005093DC00089590
:1000F0001F9318BA81E087BB19E218BB68EE73E062
:1001000080E090E0ABDF83E087BB18BB61E070E08C
:1001100080E090E0A3DF1F91089583E087BB89E230
:1001200088BB0895662391F4853011F417B83EC05A
:10013000823011F481E039C0843011F482E035C09E
:10014000833099F18A3091F58DE02FC06130A1F4B0
:10015000853011F480E929C0823011F481E925C08D
:10016000843011F482E921C0833011F483E91DC089
:100170008A30E1F48DE919C06230C1F4853011F4A0
:1001800080E813C0823011F481E80FC0843011F48C
:1001900082E80BC0833011F483E807C08A3011F481
:1001A0008DE803C08B3011F48FE887B986EC86B9EF
:1001B0003699FECF84B195B19C0140E050E0209388
:1001C000AD003093AE004093AF005093B000662373
:1001D00019F58091B5009091B600A091B700B0914B
:1001E000B800281B390B4A0B5B0B2093AD003093F2
:1001F000AE004093AF005093B00057FF08C010927C
:10020000AD001092AE001092AF001092B00020E24C
:100210003EE440E050E05AC06130A1F58091B90061
:100220009091BA00A091BB00B091BC00281B390B83
:100230004A0B5B0B2093AD003093AE004093AF00B0
:100240005093B00057FF08C01092AD001092AE005E
:100250001092AF001092B0002AE030E040E050E091
:100260006091AD007091AE008091AF009091B000B0
:10027000A5DC6093AD007093AE008093AF009093C7
:10028000B0003AC06230C1F58091BD009091BE00CF
:10029000A091BF00B091C000281B390B4A0B5B0B2B
:1002A0002093AD003093AE004093AF005093B00068
:1002B00057FF08C01092AD001092AE001092AF0030
:1002C0001092B0002CE434E040E050E06091AD00CA
:1002D0007091AE008091AF009091B0006FDC2FEF75
:1002E00033E040E050E0A2DC2093AD003093AE005C
:1002F0004093AF005093B0006091AD007091AE009C
:100300008091AF009091B00008951092B5001092C6
:10031000B6001092B7001092B80060E08AE002DFE9
:1003200084B195B1A0E0B0E08093B5009093B600A1
:10033000A093B700B093B8001092B9001092BA0021
:100340001092BB001092BC0061E08AE0EBDE84B149
:1003500095B1A0E0B0E08093B9009093BA00A0936B
:10036000BB00B093BC001092BD001092BE00109272
:10037000BF001092C00062E08AE0D4DE84B195B183
:10038000A0E0B0E08093BD009093BE00A093BF00BA
:10039000B093C000089589E288BB61E070E080E01E
:1003A00090E05CDE1092A0001092A1001092A200DA
:1003B0001092A30021C08BE288BB64E170E080E072
:1003C00090E076DE89E288BB69E170E080E090E051
:1003D00045DE8091A0009091A100A091A200B09173
:1003E000A3000196A11DB11D8093A0009093A100D0
:1003F000A093A200B093A3008091A0009091A100CF
:10040000A091A200B091A3000A97A105B1059CF2AA
:1004100008951F93182F109218010BC0BCDF6AEFCC
:1004200070E080E090E01ADE809118018F5F809389
:10043000180180911801811788F31F910895E1999F
:10044000FECF1CBA90E09FBB8EBB6DBBE29AE19AD7
:100450000895E199FECF90E09FBB8EBBE09A8DB3EB
:1004600090E0089564EF71E080E090E0F7DD93DFC5
:100470001092E6001092E7001092E8001092E90056
:100480001092B1001092B2001092B3001092B4001A
:1004900056C060E084E046DE645F7140804090407A
:1004A00014F41092C90060E084E03CDE2091660004
:1004B0003091670040916800509169002617370716
:1004C000480759074CF58091C900882329F5809188
:1004D000E6009091E700A091E800B091E900019654
:1004E000A11DB11D8093E6009093E700A093E80062
:1004F000B093E90080938000843018F083E080930B
:1005000080001092B1001092B2001092B3001092CD
:10051000B40081E08093C9008091B1009091B20055
:10052000A091B300B091B4000196A11DB11D8093BC
:10053000B1009093B200A093B300B093B400809147
:10054000B1009091B200A091B300B091B400885571
:100550009240A040B0400CF49CCF81E05ADF1BDFFA
:100560001092B1001092B2001092B3001092B40039
:1005700054C060E084E0D6DD645F7140804090400C
:1005800014F41092C90060E084E0CCDD2091660094
:100590003091670040916800509169002617370735
:1005A000480759073CF58091C900882319F58091C7
:1005B0006A0090916B00A0916C00B0916D001816CC
:1005C00019061A061B06B4F40197A109B109809314
:1005D0006A0090936B00A0936C00B0936D00109232
:1005E000B1001092B2001092B3001092B40081E0FA
:1005F0008093C9008091B1009091B200A091B300A6
:10060000B091B4000196A11DB11D8093B1009093EB
:10061000B200A093B300B093B4008091B100909168
:10062000B200A091B300B091B40088559240A040B0
:10063000B0400CF49ECF82E0ECDEADDE1092B10053
:100640001092B2001092B3001092B40054C060E057
:1006500084E068DD645F71408040904014F4109243
:10066000C90060E084E05EDD2091660030916700A3
:1006700040916800509169002617370748075907CD
:100680003CF58091C900882319F580916A0090910A
:100690006B00A0916C00B0916D008A3F9105A1059F
:1006A000B105B4F40196A11DB11D80936A00909329
:1006B0006B00A0936C00B0936D001092B10010928B
:1006C000B2001092B3001092B40081E08093C90090
:1006D0008091B1009091B200A091B300B091B400AC
:1006E0000196A11DB11D8093B1009093B200A0931B
:1006F000B300B093B4008091B1009091B200A0918A
:10070000B300B091B40088559240A040B0400CF4C2
:100710009ECF83E07EDE3FDE1092B1001092B200E9
:100720001092B3001092B40051C060E084E0FADC93
:10073000645F71408040904014F41092C90060E002
:1007400084E0F0DC20916600309167004091680001
:1007500050916900261737074807590724F58091FB
:10076000C900882301F580916E008823E1F090E0B4
:1007700069E070E011DA6AE070E045DA60936E00DB
:100780001092B1001092B2001092B3001092B40017
:100790001092DD001092DE001092DF001092E00057
:1007A00081E08093C9008091B1009091B200A09146
:1007B000B300B091B4000196A11DB11D8093B100AA
:1007C0009093B200A093B300B093B4008091B100B5
:1007D0009091B200A091B300B091B40088559240BE
:1007E000A040B0400CF4A1CF84E013DED4DD109221
:1007F000B1001092B2001092B3001092B40057C032
:1008000060E084E08FDC645F71408040904014F4CD
:100810001092C90060E084E085DC20916600309190
:100820006700409168005091690026173707480714
:10083000590754F58091C900882331F580916E00E5
:100840008F3F11F1883E50F490E06BE070E0A4D946
:100850006AE070E0D8D960936E0003C08EEF809399
:100860006E001092B1001092B2001092B30010927C
:10087000B4001092DD001092DE001092DF001092A2
:10088000E00081E08093C9008091B1009091B200B6
:10089000A091B300B091B4000196A11DB11D809349
:1008A000B1009093B200A093B300B093B4008091D4
:1008B000B1009091B200A091B300B091B4008855FE
:1008C0009240A040B0400CF49BCF6091800081E04A
:1008D000B6DD80916A0090916B00A0916C00B091A0
:1008E0006D00C297A105B10564F482E390E0A0E039
:1008F000B0E080936A0090936B00A0936C00B0937B
:100900006D0080916A0090916B00A0916C00B09195
:100910006D008B3F9105A105B10564F08AEF90E071
:10092000A0E0B0E080936A0090936B00A0936C000D
:10093000B0936D0060916A0082E081DD80916E006D
:10094000843318F484E380936E0080916E008F3FAF
:1009500019F48EEF80936E0060916E0084E06FDD7D
:1009600060918700709188008091890090918A0041
:1009700024E630E040E050E059D92093EA00622FAD
:1009800085E05DDD85E045DD06DD1092E200109238
:10099000E3001092E4001092E5001092B100109272
:1009A000B2001092B3001092B40059C08091E200DE
:1009B0009091E300A091E400B091E5000196A11DA3
:1009C000B11D8093E2009093E300A093E400B09304
:1009D000E5008D5D9540A040B040ECF06FEF80E009
:1009E0002EDD6FEF81E02BDD6FEF82E028DD6FEF12
:1009F00083E025DD6FEF84E022DD6FEF85E01FDD12
:100A0000CADCC9DCC8DCC7DCC6DCC5DCC4DCC3DCD2
:100A1000C2DCC1DCFFCF60E084E084DB20916600B3
:100A200030916700409168005091690026173707A0
:100A3000480759070CF4BACF8091B1009091B200E9
:100A4000A091B300B091B4000196A11DB11D809397
:100A5000B1009093B200A093B300B093B400809122
:100A6000B1009091B200A091B300B091B40088554C
:100A70009240A040B0407CF208956F927F928F9296
:100A80009F92AF92BF92CF92DF92EF92FF920F931D
:100A90001F9361E380E0D3DC81E0DBDC8F3F21F05A
:100AA00081E0D7DC8093800082E0D3DC8F3F69F067
:100AB00082E0CFDC90E0A0E0B0E080936A00909309
:100AC0006B00A0936C00B0936D0083E0C2DC8F3F9D
:100AD00009F46BC083E0BDDC682E77248824992458
:100AE00060926F007092700080927100909272001C
:100AF0001092DD001092DE001092DF001092E000F4
:100B0000E0906A00F0906B0000916C0010916D0015
:100B1000EE0CFF1C001F111F84E690E0A0E0B0E087
:100B2000E80EF91E0A1F1B1FE0928B00F0928C004A
:100B300000938D0010938E0025E730E040E050E0F8
:100B4000C801B7013BD8A401930138D820EE3EE29A
:100B500040E050E06BD859016A0125E230E040E006
:100B600050E0C801B7012AD864577E4080409040C9
:100B700028E730E040E050E059D8A20EB31EC41E72
:100B8000D51EA0927300B0927400C0927500D092EE
:100B9000760080918000833041F4609273007092FF
:100BA0007400809275009092760084E052DC80930D
:100BB0006E0085E04EDC8F3F91F085E04ADC90E0EE
:100BC00064E670E0E9D7AA2797FDA095BA2F809335
:100BD000870090938800A0938900B0938A0080E1F9
:100BE00038DC8F3F21F080E134DC80930B0181E120
:100BF00030DC8F3F21F081E12CDC8093100180E21A
:100C000028DC8F3F21F080E224DC8093820081E2A7
:100C100020DC8F3F21F081E21CDC8093600082E2C7
:100C200018DC8F3F21F082E214DC8093610083E2C4
:100C300010DC8F3F91F083E20CDC90E064E670E022
:100C4000ABD7AA2797FDA095BA2F809383009093E6
:100C50008400A0938500B09386001F910F91FF90B0
:100C6000EF90DF90CF90BF90AF909F908F907F904C
:100C70006F9008956F927F928F929F92AF92BF92E2
:100C8000CF92DF92EF92FF920F931F933B014C01A3
:100C90008091DD009091DE00A091DF00B091E00036
:100CA0000196A11DB11D8093DD009093DE00A093FD
:100CB000DF00B093E00083309105A105B10549F450
:100CC00060926F007092700080927100909272003A
:100CD00036C00497A105B10594F1E0906F00F09043
:100CE000700000917100109172002BE030E040E044
:100CF00050E0C801B70162D72AE030E040E050E0A0
:100D000095D726153705480559050CF41BC1C801B0
:100D1000B701F3E0660F771F881F991FFA95D1F787
:100D20006E0D7F1D801F911F2AE030E040E050E0F3
:100D30007DD762167306840695063CF503C12091A3
:100D40006F00309170004091710050917200CA01A3
:100D5000B901E2E0660F771F881F991FEA95D1F766
:100D6000620F731F841F951F660D771D881D991DC7
:100D700026E030E040E050E059D720936F003093F8
:100D800070004093710050937200E0906A00F09000
:100D90006B0000916C0010916D00EE0CFF1C001FA9
:100DA000111F84E690E0A0E0B0E0E80EF91E0A1FF3
:100DB0001B1FE0928B00F0928C0000938D0010932B
:100DC0008E0060906F007090700080907100909025
:100DD000720025E230E040E050E0C801B701EED6F5
:100DE00064577E408040904028E730E040E050E08B
:100DF0001DD759016A0125E730E040E050E0C40109
:100E0000B301DCD6A8019701D9D620EE3EE240E03E
:100E100050E00CD72A0D3B1D4C1D5D1D2093730027
:100E20003093740040937500509376002615370573
:100E30004805590544F460927300709274008092E2
:100E400075009092760097FE0CC081E090E0A0E0E3
:100E5000B0E080936F0090937000A0937100B09306
:100E6000720080916F0090917000A0917100B0911C
:100E700072008F3F9105A105B10564F08EEF90E0FF
:100E8000A0E0B0E080936F0090937000A093710099
:100E9000B093720020916F0030917000409171000A
:100EA0005091720080918F0090919000A0919100DC
:100EB000B0919200281739074A075B0799F0622F13
:100EC00083E0BDDA80916F0090917000A091710075
:100ED000B091720080938F0090939000A093910046
:100EE000B09392008091DD009091DE00A091DF0030
:100EF000B091E0000397A105B1056CF480916F00FB
:100F000090917000A0917100B0917200880F991FAC
:100F1000AA1FBB1F0FC080918000833099F480917D
:100F20006F0090917000A0917100B09172000297D3
:100F3000A109B1098093730090937400A093750088
:100F4000B09376001F910F91FF90EF90DF90CF90BC
:100F5000BF90AF909F908F907F906F900895982F43
:100F6000882339F483E08ABD80E88CBD89E288BBA0
:100F7000089581E88CBD83E28ABD81E083BF92BF82
:100F800098BD88E089BF1CBC089580E0E8DF089523
:100F90001F93182F105C812F5CDA8F5F8093FB000A
:100FA0008B3F18F08AEF8093FB006091FB00812F4C
:100FB00046DA1F9108951F9360E084E0B3D86093F0
:100FC000F4007093F5008093F6009093F700685258
:100FD000714180409040615D73408040904008F0D6
:100FE000E0C080E0D5DF8BE287BB81E088BB11E009
:100FF0001093F80018BB60ED77E080E090E02ED809
:1010000060E084E08FD86093F4007093F5008093E3
:10101000F6009093F7006E57724180409040645202
:1010200071408040904018F082E08093F80061E0C9
:1010300084E078D86093F4007093F5008093F60014
:101040009093F7006E577241804090406452714017
:101050008040904018F083E08093F80061E082E0E7
:1010600061D86093F4007093F5008093F60090933C
:10107000F7006E577241804090406452714080404A
:10108000904018F084E08093F80083E088BB61E032
:1010900070E080E090E0E2D761E082E043D86093C6
:1010A000F4007093F5008093F6009093F7006B3096
:1010B00071058105910518F085E08093F80018BB53
:1010C00061E070E080E090E0C9D718BA61E070E0BC
:1010D00080E090E0C3D761E082E024D86093F40020
:1010E0007093F5008093F6009093F700655E75426B
:1010F00080409040695572408040904018F086E0F2
:101100008093F80018BB61E070E080E090E0A6D723
:101110001092F90013C081E288BB64EF71E080E0B7
:1011200090E09CD781E088BB64EF71E080E090E0C4
:1011300095D78091F9008F5F8093F9009091F80026
:101140008091F900891738F39130B9F06CED75E0B2
:1011500080E090E083D781E288BB6091F4007091D9
:10116000F5008091F6009091F70078D781E088BB78
:1011700060ED77E080E090E071D76091820080E2DE
:101180005ED96091600081E25AD96091610082E28B
:1011900056D98091830064E62AD5682F83E24FD91F
:1011A00026CF1F9108952F923F924F925F926F9298
:1011B0007F928F929F92AF92BF92CF92DF92EF92E7
:1011C000FF920F931F9319E218BB61E070E080E07B
:1011D00090E044D78BE288BB61E070E080E090E073
:1011E0003DD761E082E09ED728EE33E040E050E05A
:1011F000E5D422E03BE040E050E018D52093980091
:101200003093990040939A0050939B0018BB2B3F5A
:101210003105410551053CF018BB82E0B9DE81E1A2
:101220008093930073C081E09ADE809161001091F9
:101230006E00813009F049C0812F8695282E332415
:10124000442455242091F0003091F1004091F200A7
:101250005091F300612E772488249924EE24FF24F2
:101260008701AA24BB24650115C0C601B501661912
:1012700077098809990924E630E040E050E0D6D4A7
:10128000220D331D441D551D28BD0894E11CF11C81
:10129000011D111DA60CB71CC81CD91C83E3E81640
:1012A000F104010511050CF32093F0003093F100D7
:1012B0004093F2005093F300E092EC00F092ED00C6
:1012C0000093EE001093EF0021C0612F70E080E0EA
:1012D00090E02091EC003091ED004091EE005091B3
:1012E000EF006CD424E630E040E050E09FD4812F42
:1012F0008695280F311D411D511D2093F00030931C
:10130000F1004093F2005093F30018BD1F910F912C
:10131000FF90EF90DF90CF90BF90AF909F908F9015
:101320007F906F905F904F903F902F90089589E24B
:1013300088BB61E070E080E090E090D660E083E000
:10134000F1D624E030E040E050E070D42093FD007E
:101350003093FE004093FF005093000160E085E071
:10136000E1D624E030E040E050E060D42093010179
:101370003093020140930301509304018091FD00DA
:101380009091FE00A091FF00B09100018C3261E0CD
:10139000960760E0A60760E0B60774F42C3261E0BF
:1013A000360760E0460760E0560734F481E080933A
:1013B000050181E090E00895255F314040405040B4
:1013C0001CF083E090E00895855F9140A040B0401C
:1013D0001CF082E090E0089581E090E0089589E2B9
:1013E00088BB61E070E080E090E038D660E083E0A8
:1013F00099D624E030E040E050E018D42093FD007E
:101400003093FE004093FF005093000190E0295B71
:101410003B40404050400CF091E081E09827892FFC
:1014200090E00895EF92FF920F931F9360ED77E0A5
:1014300080E090E013D681E08093930080937F005A
:1014400064D760E084E06ED6655F71408040904074
:101450001CF084E08093930010DB4AD613E017BBA6
:1014600089E288BB60E082E05DD69B01AC016093BD
:101470009C0070939D0080939E0090939F00283560
:101480008BE1380780E0480780E058071CF482E0D1
:101490008093930021583E434040504024F081E027
:1014A00077DD109393008091870090918800A09140
:1014B0008900B0918A000097A105B10559F460E058
:1014C00082E030D660938700709388008093890013
:1014D00090938A008091830090918400A091850070
:1014E000B09186000097A105B10541F08093870077
:1014F00090938800A0938900B0938A00E0908700C1
:10150000F09088000091890010918A0020E530E079
:1015100040E050E0C801B70151D324E630E040E09C
:1015200050E084D3209366003093670040936800B6
:101530005093690025E530E040E050E0C801B70174
:101540003DD324E630E040E050E070D320936200C9
:10155000309363004093640050936500E8DE80930D
:10156000FC001092D1001092D2001092D300109281
:10157000D40019C064EF71E080E090E06FD50BD724
:101580008091D1009091D200A091D300B091D4006D
:101590000196A11DB11D8093D1009093D200A0931C
:1015A000D300B093D4008091930090E0A0E0B0E02D
:1015B0002091D1003091D2004091D3005091D400BD
:1015C000281739074A075B07ACF2F5DC80919300D6
:1015D0008230F0F71092B1001092B2001092B30076
:1015E0001092B4001CC060E084E09CD569557B413A
:1015F000804090400CF036D78091B1009091B200BD
:10160000A091B300B091B4000196A11DB11D8093CB
:10161000B1009093B200A093B300B093B400809156
:10162000B1009091B200A091B300B091B400815A82
:101630009440A040B040BCF280918200882319F011
:1016400083E080938000A7D6A6D6A5D6A4D68091A5
:101650000501882321F09FD69ED69DD69CD68091E9
:10166000CA009091CB00A091CC00B091CD00019622
:10167000A11DB11D8093CA009093CB00A093CC0014
:10168000B093CD008091070190910801A0910901CC
:10169000B0910A010196A11DB11D8093070190939D
:1016A0000801A0930901B0930A016FDC8091190130
:1016B00090911A01892B61F092DE882349F46CED38
:1016C00075E080E090E0CAD410921A0110921901DE
:1016D00060E084E027D59B01AC0160939400709397
:1016E000950080939600909397008091660090916A
:1016F0006700A0916800B091690082179307A40762
:10170000B507ECF58091C9008823C9F580910501E2
:101710008823A9F48091620090916300A0916400F5
:10172000B0916500281739074A075B076CF4809170
:10173000EB008F5F8093EB008330E8F4B6C0F7DDF9
:101740008093FC00813019F41092EB00AEC09091B0
:10175000EB009F5F9093EB00833039F4933008F4F3
:10176000A4C080E18093930065C1823009F09DC0E0
:10177000933008F49AC080E18093930096C0245F70
:101780003140404050406CF41092C90081E0809399
:101790007F001092CA001092CB001092CC001092E1
:1017A000CD008091CA009091CB00A091CC00B09167
:1017B000CD00833A9105A105B10584F08091C9005F
:1017C000813061F480918000833041F0809160002D
:1017D000813021F482E080937F0067C08091060110
:1017E000882309F03CCF8091C1009091C200A09164
:1017F000C300B091C4008D529140A040B04008F4A5
:101800002ECF8091070190910801A0910901B0911C
:101810000A01895E9340A040B0400CF420CF809133
:10182000830090918400A0918500B091860000977C
:10183000A105B10509F413CF60E082E073D47B0108
:101840008C01609387007093880080938900909347
:101850008A0020E530E040E050E0B0D124E630E0FE
:1018600040E050E0E3D1209366003093670040935E
:1018700068005093690025E530E040E050E0C80181
:10188000B7019CD124E630E040E050E0CFD1209376
:10189000620030936300409364005093650084E0DD
:1018A00077DB81E080930601DACE99DD882309F4A5
:1018B000D6CE8091190190911A014E9708F0CFCEA3
:1018C00080911101813009F4B5C06DDC61E070E0F8
:1018D00080E090E0C3D31092C5001092C600109231
:1018E000C7001092C8008091C1009091C200A091E1
:1018F000C300B091C4000196A11DB11D8093C10029
:101900009093C200A093C300B093C4008091C5001F
:101910009091C600A091C700B091C8000196A11D8A
:10192000B11D8093C5009093C600A093C700B093EB
:10193000C80061E084E0F6D3609394007093950052
:101940008093960090939700685B7B408040904026
:101950008CF480918000813021F080917F00823072
:1019600021F481E080937F0065C08091C9008823C5
:1019700009F460C080917F00823021F08091800066
:101980008130B1F5E0906F00F0907000009171002F
:1019900010917200C801B70122E030E040E050E051
:1019A00045D1E20EF31E041F151F8091C5009091D2
:1019B000C600A091C700B091C800E816F9060A0752
:1019C0001B070CF0A3CF8091190190911A01019689
:1019D00090931A01809319011092C5001092C600CD
:1019E0001092C7001092C8004E9708F48FCF22C003
:1019F0002091C5003091C6004091C7005091C800A9
:101A00008091730090917400A0917500B091760060
:101A100082179307A407B5070CF078CF81E0809375
:101A2000C9008091190190911A01039690931A01AF
:101A300080931901AADA32D36BE470E080E090E081
:101A40000DD389E288BB8091C900882391F48091ED
:101A5000190190911A01019690931A01809319012E
:101A60006091C5007091C6008091C7009091C80038
:101A700001D962E08BE056D324E630E040E050E04C
:101A80009DD068567447804090402DE630E040E09D
:101A900050E0CCD020930C0130930D0140930E0107
:101AA00050930F012C333105410551052CF083E093
:101AB0006FDA81E08093110120910C0130910D01CA
:101AC00040910E0150910F01283331054105510518
:101AD00014F41092110180911101813019F482E106
:101AE000809393001092CA001092CB001092CC0009
:101AF0001092CD0010920701109208011092090176
:101B000010920A0180910B0190E0A0E0B0E08217F2
:101B10009307A407B5072CF420930B01622F80E1F3
:101B20008ED4609198007091990080919A00909164
:101B30009B002AE030E040E050E078D08091100136
:101B400090E0A0E0B0E082179307A407B5072CF45B
:101B500020931001622F81E172D480919300882339
:101B600009F47DCD64E670E080E090E077D280916A
:101B70009300803111F481E04CD480919300813145
:101B800011F482E046D480919300823111F483E015
:101B900040D41092930063CD5527002480FF02C0EB
:101BA000060E571F660F771F6115710521F0969578
:101BB0008795009799F7952F802D0895FF27EE2799
:101BC000BB27AA2760FF04C0A20FB31FE41FF51FA5
:101BD000220F331F441F551F96958795779567955C
:101BE00089F70097760771F7CF01BD010895991B1A
:101BF00079E004C0991F961708F0961B881F7A9504
:101C0000C9F78095089597FB092E07260AD077FD1E
:101C100004D027D006D000201AF4709561957F4F2C
:101C20000895F6F7909581959F4F089597FB092E9B
:101C300005260ED057FD04D028D00AD0001C38F459
:101C400050954095309521953F4F4F4F5F4F0895E8
:101C5000F6F790958095709561957F4F8F4F9F4FC8
:101C60000895AA1BBB1B51E107C0AA1FBB1FA617E3
:101C7000B70710F0A61BB70B881F991F5A95A9F735
:101C800080959095BC01CD010895A1E21A2EAA1B62
:101C9000BB1BFD010DC0AA1FBB1FEE1FFF1FA2171C
:101CA000B307E407F50720F0A21BB30BE40BF50B19
:101CB000661F771F881F991F1A9469F760957095A2
:101CC000809590959B01AC01BD01CF010895FFCF98
:101CD00001017C1500007017000050000000FE4656
:101CE000000000CD000000640000000100000001C1
:021CF0000200F0
:00000001FF
